:1000000000308A0066280000D3346D38EC32202A94
:10001000E832F236EF36653AE8327200A83129103C
:10002000CB306B36E9352019B018B3060A00F73B20
:1000300077176D366131AE31FA060A008316031761
:100040008C170C140000000083120C087F39031970
:1000500064280313A10003170D080313A20003175C
:100060000F080313A30021080C1E3428990022084E
:1000700003178D000313230803178F0083168C17B3
:100080000C140000000083120C0D0E0D7F390319B3
:1000900064280313A10003170D080313A20003171C
:1000A0000F080313A30021080C1E542899002208EE
:1000B00003178D000313230803178F008D0A0319FC
:1000C0008F0A03131E2803170313080084018313E8
:1000D0001F308305713083168F000F0803178711B7
:1000E0000C3003139900A2309800903083129800CE
:1000F000831603170908C039890003131F129F12C2
:100100000030031788008312870188018901FF30BE
:100110000313A000831603170908C03989000313CD
:100120001F129F12003003178800831203131F133E
:100130009F1383169F1383121F149412A01220087A
:1001400083168700831220162008831687008312E7
:10015000A01120088316870001308312940000301C
:10016000831694000108C739083881008312900172
:100170000030F800920000308316920083122015A0
:100180002008831687008312970183169B019C0128
:1001900001309D00831203178701880189017130A6
:1001A000831603138F000F080430831203178D008A
:1001B00000308F0003131E200E3003178D00003017
:1001C0008F0003131E20173003178D0000308F009F
:0801D00003131E20EA2863005E
:04400E00F52CFF3F4F
:00000001FF
